:20000000B67E80840FBDEE9CA600BDF9A49683849F8A409783B77A00CE0000BDF992CE001D
:2000200002BDF9927EF999CE0100DF8DDF8B7F008F39AC7358403A1D0F0805050403020240
:2000400002017D008F271ADE8BA600847F9A92B77A017A008F088C010C2603CE0100DF8BD4
:20006000399683849F9783B77A003900000000000000000000000000000000000000000087
:20008000000000000000000000000000000000000000000000000000000000000000000060
:2000A000000000000000000000000000000000000000000000000000000000000000000040
:2000C0000000000000000000000000000000008FCE00B38680C6088D4BCE00BBC6084F8D31
:2000E00043CEECECDF93CEF7E4DFA19600261BCEED87DF95CEF9DDDF97CEFA20DF99CEF4B3
:20010000A6DF9BCEE6C5DF9D2003BDE0C3CE0000DFCBDFCDCE0000BDF992CE0002BDF992F5
:200120000E7EF92BA700085A2EFA39DECBA6B32A33088C000826F67F00CCF67802C50226E6
:20014000EAC634F77801C63CF77801CE0000A6BB270A6ABB2606A6B3847FA7B3088C0008D6
:2001600026EC20C7DFCBDFCD16847CA7B3A6C37800CEDECDC501270EC5022706368D1A3268
:20018000DECDEEA32002EE93C430AD00DECB20A1A7C3A6B3847FA7B339DECBA6B38A80A769
:2001A000B36FBB39DECBE6B3CA81A7BB2602C47FE7B33233DFCD7800CEDECDA7A3E7A43925
:2001C000DECBE6B3CA8320E8DECB36A6B384CFC4301BA7B33239DECBE6B3C43039BDFA63A0
:2001E0005D2B3CCE00034D2A0ED65C2708E6B3C4FEE7B32002847F7EF990A60016D80FD7E9
:200200000F088C03802603CE01104D2A0DE600D7D3088C03802603CE0110DFCF7F00D43943
:2002200036BDF999324D2A1B847FD6D3C51026EFC560270CD65C270837BDFB8B327EEF2DE0
:200240007EEEF5C650D7D6856027F5915527F1BDEEF57A00D627C8BDFA635D2BC24D2AE7DA
:200260007EFA28DECF9CD12713BDF9FA7D00152F09BDE86FD615C50227025F39C68039CE3C
:200280000110DFD1DFCF39F67A002A028D10F67C002A0AF6E670C1AA2603BDE8AE3BC501A3
:2002A0002758B67A01847FC4702709C5102703D7D7398A807D00D727047F00D7397D00D4D8
:2002C0002B31DED1A700088C03802603CE0110DFD14D2A0DE700088C03802603CE0110DF34
:2002E000D1088C03802603CE01109CCF2604868097D439868097D57EFB8BC502270B968347
:200300008460812026037EF842C5042703B67A0139868097289664851027037EEFB07EEF12
:20032000D07F00283986809729397F002939965184BF200496518A40975139BDF9C08146D0
:2003400026069651847F20F0814826EE96518A8020E68680972A397F002A398680972D39BE
:200360007F002D397D005226147D0015260F966085202609B6780284048A809752397F009B
:2003800052398602972E397F002E39B6780384F7B778038A08B7780339BDF9C0BDF35E8A7D
:2003A000907EEF2DD6CCC1012604D6632B4DBDF9C07F0074812E260786109774BDF9C0BDBB
:2003C000F35E25389B749774BDF9C0BDF35E484848489773BDF9C0BDF35E2520CE0055DFDC
:2003E000CDD674DBCED7CED6CDC900D7CDDECDD6731BA700D6002703BDE094397EFB8BBDA7
:20040000F9C036BDFDAA32812126037EE90081302D6126028D0D813926028D2E81382602A6
:200420008D3B39DE53C6108D58DFD88D51CE0055C6108D4D8D488D46DED8C60E8D438D3E9A
:20044000CE0065C60E8D3A8D3539CEEBC7C6028D308D2BCEEB19C6028D278D2239B67E00AC
:200460008D3F8D1AB679008D388D13B67D008D318D0C398DAE8D078DD18D038DE0397EF0E1
:200480006ADFCD37A60036BDF379BDEF2D32BDF37DBDEF2DBDF04733DECD08DFCD5A26E112
:2004A0003997D8C608D7D9BDF0477400D8240486462002864EBDEF2D7A00D926EA398601F0
:2004C0002006868020028611F6E670C1AA261BF67900C58026147EE671F6E670C1AA260A95
:2004E000F67900C58026037EE82239FEE0008C544A26F77EE03E86027EEF2D860320F9BD1C
:20050000F9C080209773BDF9C09155270A36BDEF16327A00732EF6398620D665C580270525
:20052000965D20014FD665C50227037F00299A2936BDEEAB96522A358404F67802C404111D
:20054000262B32D62337D62437D62637D6273736BDF3B5BDFDD3BDF3B53233F77F0CD727DE
:2005600033F77F0DD72633D72433D72336BDFDD6317EEFD0D665C50427304F3620338D0F6A
:2005800036202ED665C50427F58D0F8D02201E8620D665C5402702965D39962F2A07966225
:2005A0002A03BDF2583986A020038DEE4F367F00287F0029BDEEAB965227128404F67802C7
:2005C000C404112603BDF3B58D09BDF3B58D04317EEFD0BDF026D621CB07867FD7D897D9FA
:2005E0009625BDF3418B4FD921D7DA97DB30E602DE2396282A08B7700001A5002606B7702F
:200600000001E7009CDA270D9CD827030820E3DE21DF2320DD7EF34F8620D665C580270292
:20062000965DBDEEABD665C50127037F00299A29C650D027D7DBDE23D6282A08B7700001C3
:20064000E6002B0CB7700001A700087A00DB26E8DE23B7700001A60095282703BDF1513955
:200660004F20BF965D20BEBDFB2ADE238650902797DBC620B7700001A6009528260DB770CE
:200680000001E70016087A00DB26E9DE2339BDFB2ADE23C64FF07F092714B7700001A6013C
:2006A0009528260AB7700001A700085A20EA965DB7700001A700397D00282701397F002969
:2006C000BDF03CDE23DFDC96522A3DF678028404C404112633C6874D2602CB0886D0D7DC5E
:2006E00097DDDEDCA604364A2A028617A70432BDF341EB00D77D977E9625BDF341DB21D738
:200700007F9780C650BDF4129625912627424D27244A97DABDF341DB21D7D897D9DED8C6B4
:2007200050B7700001A600B7700001A750085A26F096DA20D5DE21DF7D967E8B30978096C8
:200740007D8907977FC650BDF412861797DA20BA965D7EFE257D00282701397F0029BDF0C6
:200760003C96269125273C81172616D621CB078630D77D977EDE21DF7FC650BDF4124F2007
:20078000E236BDF341DB21D7D897D9DED8C650B7700001A650B7700001A700085A26F032D2
:2007A0004C20C0BDF341DB21D77DD7D8977E97D996522733F67802C40484041126298804AA
:2007C000488B87C6D0977FD780DE7FA6044C81172F014FA704BDF341EB00D77F9780DE7F01
:2007E000DFD8C650BDF412DED8C650965DB7700001A700085A26F639FA87E900FA87E90050
:00000001FF
